BL51 BANKED LINKER/LOCATER V5.00                                                        05/05/2011  10:22:17  PAGE 1


BL51 BANKED LINKER/LOCATER V5.00, INVOKED BY:
C:\KEIL中文版\KEIL\C51\BIN\BL51.EXE Function2.obj TO Function RAMSIZE (256)


MEMORY MODEL: SMALL


INPUT MODULES INCLUDED:
  Function2.obj (FUNCTION2)
  C:\KEIL中文版\KEIL\C51\LIB\C51S.LIB (?C_STARTUP)
  C:\KEIL中文版\KEIL\C51\LIB\C51S.LIB (?C_INIT)


LINK MAP OF MODULE:  Function (FUNCTION2)


            TYPE    BASE      LENGTH    RELOCATION   SEGMENT NAME
            -----------------------------------------------------

            * * * * * * *   D A T A   M E M O R Y   * * * * * * *
            REG     0000H     0008H     ABSOLUTE     "REG BANK 0"
                    0008H     0018H                  *** GAP ***
            BIT     0020H.0   0000H.1   UNIT         ?BI?BUSYTEST?FUNCTION2
                    0020H.1   0000H.7                *** GAP ***
            DATA    0021H     001AH     UNIT         ?DT?FUNCTION2
            IDATA   003BH     0001H     UNIT         ?STACK

            * * * * * * *   C O D E   M E M O R Y   * * * * * * *
            CODE    0000H     0003H     ABSOLUTE     
                    0003H     0008H                  *** GAP ***
            CODE    000BH     0003H     ABSOLUTE     
            CODE    000EH     0224H     UNIT         ?CO?FUNCTION2
            CODE    0232H     0094H     UNIT         ?PR?SETFRE?FUNCTION2
            CODE    02C6H     008CH     UNIT         ?C_C51STARTUP
            CODE    0352H     008AH     UNIT         ?PR?TIME0?FUNCTION2
            CODE    03DCH     0078H     UNIT         ?PR?_WRITE_HANSHU?FUNCTION2
            CODE    0454H     0076H     UNIT         ?PR?KEYSCAN?FUNCTION2
            CODE    04CAH     0066H     UNIT         ?PR?LCDINIT?FUNCTION2
            CODE    0530H     005AH     UNIT         ?PR?MAIN?FUNCTION2
            CODE    058AH     0023H     UNIT         ?PR?_WRITEDAT?FUNCTION2
            CODE    05ADH     001FH     UNIT         ?PR?_WRITECOM?FUNCTION2
            CODE    05CCH     0018H     UNIT         ?PR?_DELAYMS?FUNCTION2
            CODE    05E4H     0017H     UNIT         ?PR?BUSYTEST?FUNCTION2
            CODE    05FBH     0015H     UNIT         ?PR?_WRITE_FRE?FUNCTION2
            CODE    0610H     0012H     UNIT         ?PR?_DELAY?FUNCTION2
            CODE    0622H     0012H     UNIT         ?PR?KEYDOWN?FUNCTION2
            CODE    0634H     0010H     UNIT         ?C_INITSEG



OVERLAY MAP OF MODULE:   Function (FUNCTION2)


SEGMENT
  +--> CALLED SEGMENT
---------------------
?PR?TIME0?FUNCTION2
  +--> ?CO?FUNCTION2
BL51 BANKED LINKER/LOCATER V5.00                                                      05/05/2011  10:22:17  PAGE 2



*** NEW ROOT ***************************************************

?C_C51STARTUP
  +--> ?PR?MAIN?FUNCTION2
  +--> ?C_INITSEG

?PR?MAIN?FUNCTION2
  +--> ?PR?LCDINIT?FUNCTION2
  +--> ?PR?KEYDOWN?FUNCTION2
  +--> ?PR?SETFRE?FUNCTION2
  +--> ?PR?_WRITE_HANSHU?FUNCTION2

?PR?LCDINIT?FUNCTION2
  +--> ?PR?_DELAYMS?FUNCTION2
  +--> ?PR?_WRITECOM?FUNCTION2
  +--> ?CO?FUNCTION2
  +--> ?PR?_WRITEDAT?FUNCTION2

?PR?_DELAYMS?FUNCTION2
  +--> ?PR?_WRITECOM?FUNCTION2

?PR?KEYDOWN?FUNCTION2
  +--> ?PR?KEYSCAN?FUNCTION2

?PR?KEYSCAN?FUNCTION2
  +--> ?PR?_DELAY?FUNCTION2

?PR?SETFRE?FUNCTION2
  +--> ?PR?KEYDOWN?FUNCTION2
  +--> ?PR?_WRITE_FRE?FUNCTION2

?PR?_WRITE_FRE?FUNCTION2
  +--> ?PR?_WRITECOM?FUNCTION2
  +--> ?CO?FUNCTION2
  +--> ?PR?_WRITEDAT?FUNCTION2

?PR?_WRITE_HANSHU?FUNCTION2
  +--> ?PR?_WRITECOM?FUNCTION2
  +--> ?CO?FUNCTION2
  +--> ?PR?_WRITEDAT?FUNCTION2
  +--> ?PR?_DELAYMS?FUNCTION2



SYMBOL TABLE OF MODULE:  Function (FUNCTION2)

  VALUE           TYPE          NAME
  ----------------------------------

  -------         MODULE        FUNCTION2
  C:0000H         SYMBOL        _ICE_DUMMY_
  D:0080H         PUBLIC        P0
  D:0090H         PUBLIC        P1
  D:00A0H         PUBLIC        P2
  D:00B0H         PUBLIC        P3
  B:00B0H.4       PUBLIC        T0
BL51 BANKED LINKER/LOCATER V5.00                                                      05/05/2011  10:22:17  PAGE 3


  B:00D0H.6       PUBLIC        AC
  B:00B0H.5       PUBLIC        T1
  C:0622H         PUBLIC        keydown
  B:00A8H.7       PUBLIC        EA
  C:05E4H         PUBLIC        busytest
  B:00B0H.5       PUBLIC        lcden
  C:0019H         PUBLIC        str1
  D:0021H         PUBLIC        k_old
  C:05FBH         PUBLIC        _write_Fre
  C:001DH         PUBLIC        str2
  C:0021H         PUBLIC        str3
  C:0025H         PUBLIC        str4
  C:0029H         PUBLIC        str5
  C:002EH         PUBLIC        str6
  B:00B0H.7       PUBLIC        RD
  B:00A8H.4       PUBLIC        ES
  B:00B0H.7       PUBLIC        lcdrs
  B:0098H.0       PUBLIC        RI
  D:0022H         PUBLIC        flag
  B:00B0H.2       PUBLIC        INT0
  B:00D0H.7       PUBLIC        CY
  D:0023H         PUBLIC        keynum
  B:0098H.1       PUBLIC        TI
  B:00B0H.3       PUBLIC        INT1
  B:00B0H.6       PUBLIC        lcdrw
  B:00B8H.4       PUBLIC        PS
  B:00D0H.2       PUBLIC        OV
  C:0530H         PUBLIC        main
  D:0024H         PUBLIC        nian
  D:0025H         PUBLIC        miao
  B:00B0H.6       PUBLIC        WR
  D:0026H         PUBLIC        time
  D:0089H         PUBLIC        TMOD
  C:000EH         PUBLIC        tab
  D:0027H         PUBLIC        temp
  D:0028H         PUBLIC        fen
  D:0029H         PUBLIC        fre
  B:0088H.1       PUBLIC        IE0
  B:0088H.3       PUBLIC        IE1
  C:0352H         PUBLIC        Time0
  D:002AH         PUBLIC        shi
  D:002BH         PUBLIC        zhou
  C:058EH         PUBLIC        _writedat
  B:00A8H.1       PUBLIC        ET0
  D:002CH         PUBLIC        key
  B:00A8H.3       PUBLIC        ET1
  B:0088H.5       PUBLIC        TF0
  B:0088H.7       PUBLIC        TF1
  C:0232H         PUBLIC        SetFre
  B:0098H.2       PUBLIC        RB8
  D:008CH         PUBLIC        TH0
  B:00A8H.0       PUBLIC        EX0
  B:0088H.0       PUBLIC        IT0
  B:0098H.3       PUBLIC        TB8
  B:00A8H.2       PUBLIC        EX1
  B:0088H.2       PUBLIC        IT1
  C:05ADH         PUBLIC        _writecom
BL51 BANKED LINKER/LOCATER V5.00                                                      05/05/2011  10:22:17  PAGE 4


  B:00D0H.0       PUBLIC        P
  B:0098H.7       PUBLIC        SM0
  D:008AH         PUBLIC        TL0
  B:0098H.6       PUBLIC        SM1
  B:0098H.5       PUBLIC        SM2
  C:05D6H         PUBLIC        _delayms
  D:002DH         PUBLIC        yue
  B:00B8H.1       PUBLIC        PT0
  B:00B8H.3       PUBLIC        PT1
  B:00D0H.3       PUBLIC        RS0
  B:0088H.4       PUBLIC        TR0
  B:00D0H.4       PUBLIC        RS1
  B:0088H.6       PUBLIC        TR1
  B:00B8H.0       PUBLIC        PX0
  B:00B8H.2       PUBLIC        PX1
  D:002EH         PUBLIC        ri
  D:002FH         PUBLIC        a
  D:0030H         PUBLIC        b
  C:0032H         PUBLIC        sin_tab
  B:0098H.4       PUBLIC        REN
  D:0031H         PUBLIC        h
  D:0032H         PUBLIC        i
  C:0132H         PUBLIC        tri_tab
  D:0033H         PUBLIC        j
  D:0034H         PUBLIC        k
  C:04CAH         PUBLIC        lcdinit
  D:0035H         PUBLIC        m
  D:0036H         PUBLIC        n
  B:00B0H.0       PUBLIC        RXD
  D:0037H         PUBLIC        q
  D:0039H         PUBLIC        fangbo
  B:00B0H.1       PUBLIC        TXD
  C:0610H         PUBLIC        _delay
  C:0454H         PUBLIC        keyscan
  D:003AH         PUBLIC        t
  B:00D0H.5       PUBLIC        F0
  C:03DCH         PUBLIC        _write_hanshu
  B:0080H.7       PUBLIC        lcdbf
  -------         PROC          _DELAY
  D:0007H         SYMBOL        x
  -------         DO            
  D:0006H         SYMBOL        j
  -------         ENDDO         
  C:0610H         LINE#         103
  C:0610H         LINE#         104
  C:0610H         LINE#         105
  C:0616H         LINE#         106
  C:061EH         LINE#         107
  C:0621H         LINE#         108
  C:0621H         LINE#         109
  -------         ENDPROC       _DELAY
  C:05CFH         SYMBOL        L?0116
  C:05D1H         SYMBOL        L?0117
  -------         PROC          L?0115
  -------         ENDPROC       L?0115
  C:05CFH         SYMBOL        L?0116
  C:05D1H         SYMBOL        L?0117
BL51 BANKED LINKER/LOCATER V5.00                                                      05/05/2011  10:22:17  PAGE 5


  -------         PROC          _DELAYMS
  D:0007H         SYMBOL        xms
  -------         DO            
  D:0007H         SYMBOL        i
  D:0006H         SYMBOL        j
  -------         ENDDO         
  C:05D6H         LINE#         111
  C:05D6H         LINE#         112
  C:05D6H         LINE#         114
  C:05DCH         LINE#         115
  C:05E3H         LINE#         117
  -------         ENDPROC       _DELAYMS
  -------         PROC          BUSYTEST
  -------         DO            
  B:0020H.0       SYMBOL        presence
  -------         ENDDO         
  C:05E4H         LINE#         119
  C:05E4H         LINE#         120
  C:05E4H         LINE#         122
  C:05E6H         LINE#         123
  C:05E8H         LINE#         124
  C:05EAH         LINE#         125
  C:05F0H         LINE#         126
  C:05F4H         LINE#         127
  C:05F5H         LINE#         128
  C:05F6H         LINE#         129
  C:05F8H         LINE#         130
  C:05FAH         LINE#         132
  -------         ENDPROC       BUSYTEST
  -------         PROC          _WRITECOM
  D:0007H         SYMBOL        com
  C:05ADH         LINE#         134
  C:05ADH         LINE#         135
  C:05ADH         LINE#         137
  C:05AFH         LINE#         138
  C:05B1H         LINE#         139
  C:05B3H         LINE#         140
  C:05B9H         LINE#         141
  C:05BBH         LINE#         142
  C:05C1H         LINE#         143
  C:05C3H         LINE#         144
  C:05C9H         LINE#         145
  C:05CBH         LINE#         147
  -------         ENDPROC       _WRITECOM
  -------         PROC          L?0118
  -------         ENDPROC       L?0118
  -------         PROC          _WRITEDAT
  D:0007H         SYMBOL        dat
  C:058EH         LINE#         150
  C:058EH         LINE#         151
  C:058EH         LINE#         153
  C:0590H         LINE#         154
  C:0592H         LINE#         155
  C:0594H         LINE#         156
  C:059AH         LINE#         158
  C:059CH         LINE#         159
  C:05A2H         LINE#         160
BL51 BANKED LINKER/LOCATER V5.00                                                      05/05/2011  10:22:17  PAGE 6


  C:05A4H         LINE#         161
  C:05AAH         LINE#         162
  C:05ACH         LINE#         164
  -------         ENDPROC       _WRITEDAT
  -------         PROC          _WRITE_HANSHU
  D:0005H         SYMBOL        d
  C:03DCH         LINE#         166
  C:03DEH         LINE#         167
  C:03DEH         LINE#         168
  C:03E3H         LINE#         169
  C:03E6H         LINE#         170
  C:03E9H         LINE#         171
  C:03E9H         LINE#         172
  C:03EFH         LINE#         173
  C:03F4H         LINE#         174
  C:03FDH         LINE#         175
  C:03FDH         LINE#         176
  C:0400H         LINE#         177
  C:0403H         LINE#         178
  C:0403H         LINE#         179
  C:0409H         LINE#         180
  C:040EH         LINE#         181
  C:0417H         LINE#         182
  C:0417H         LINE#         183
  C:041AH         LINE#         184
  C:041DH         LINE#         185
  C:041DH         LINE#         186
  C:0427H         LINE#         187
  C:042CH         LINE#         188
  C:0435H         LINE#         189
  C:0435H         LINE#         190
  C:0438H         LINE#         191
  C:043BH         LINE#         192
  C:043BH         LINE#         193
  C:0445H         LINE#         194
  C:044AH         LINE#         195
  C:0453H         LINE#         196
  C:0453H         LINE#         197
  -------         ENDPROC       _WRITE_HANSHU
  -------         PROC          _WRITE_FRE
  D:0006H         SYMBOL        d
  C:05FBH         LINE#         199
  C:05FDH         LINE#         200
  C:05FDH         LINE#         201
  C:0602H         LINE#         203
  C:060BH         LINE#         204
  -------         ENDPROC       _WRITE_FRE
  -------         PROC          LCDINIT
  C:04CAH         LINE#         208
  C:04CAH         LINE#         209
  C:04CAH         LINE#         210
  C:04CCH         LINE#         211
  C:04CCH         LINE#         212
  C:04CFH         LINE#         213
  C:04CFH         LINE#         214
  C:04CFH         LINE#         215
  C:04CFH         LINE#         216
BL51 BANKED LINKER/LOCATER V5.00                                                      05/05/2011  10:22:17  PAGE 7


  C:04D2H         LINE#         217
  C:04D4H         LINE#         218
  C:04D7H         LINE#         219
  C:04DCH         LINE#         220
  C:04E0H         LINE#         221
  C:04E2H         LINE#         222
  C:04E5H         LINE#         223
  C:04E7H         LINE#         224
  C:04EAH         LINE#         225
  C:04ECH         LINE#         226
  C:04EFH         LINE#         235
  C:04F1H         LINE#         236
  C:04F4H         LINE#         238
  C:04F7H         LINE#         239
  C:04F7H         LINE#         240
  C:0501H         LINE#         241
  C:0506H         LINE#         242
  C:050FH         LINE#         245
  C:0511H         LINE#         246
  C:0514H         LINE#         248
  C:0517H         LINE#         249
  C:0517H         LINE#         250
  C:0521H         LINE#         251
  C:0526H         LINE#         252
  C:052FH         LINE#         278
  -------         ENDPROC       LCDINIT
  -------         PROC          MAIN
  C:0530H         LINE#         281
  C:0530H         LINE#         282
  C:0530H         LINE#         283
  C:0533H         LINE#         284
  C:0536H         LINE#         285
  C:0538H         LINE#         286
  C:053BH         LINE#         287
  C:053EH         LINE#         288
  C:0540H         LINE#         289
  C:0542H         LINE#         290
  C:0544H         LINE#         291
  C:0546H         LINE#         292
  C:0549H         LINE#         297
  C:0549H         LINE#         298
  C:0549H         LINE#         299
  C:054CH         LINE#         300
  C:0551H         LINE#         301
  C:0551H         LINE#         302
  C:0553H         LINE#         303
  C:0555H         LINE#         304
  C:0557H         LINE#         305
  C:055AH         LINE#         306
  C:055CH         LINE#         307
  C:055EH         LINE#         308
  C:0560H         LINE#         309
  C:0560H         LINE#         310
  C:056AH         LINE#         311
  C:0574H         LINE#         312
  C:057EH         LINE#         313
  C:0588H         LINE#         314
BL51 BANKED LINKER/LOCATER V5.00                                                      05/05/2011  10:22:17  PAGE 8


  -------         ENDPROC       MAIN
  -------         PROC          SETFRE
  C:0232H         LINE#         320
  C:0232H         LINE#         321
  C:0232H         LINE#         323
  C:0235H         LINE#         325
  C:0245H         LINE#         326
  C:0255H         LINE#         327
  C:0265H         LINE#         328
  C:0275H         LINE#         329
  C:0285H         LINE#         330
  C:0295H         LINE#         331
  C:02A5H         LINE#         332
  C:02B5H         LINE#         333
  C:02C5H         LINE#         337
  -------         ENDPROC       SETFRE
  -------         PROC          KEYSCAN
  C:0454H         LINE#         341
  C:0454H         LINE#         342
  C:0454H         LINE#         343
  C:0457H         LINE#         344
  C:045CH         LINE#         345
  C:045FH         LINE#         346
  C:0462H         LINE#         347
  C:0469H         LINE#         348
  C:046CH         LINE#         349
  C:0471H         LINE#         350
  C:0476H         LINE#         351
  C:047BH         LINE#         352
  C:0480H         LINE#         353
  C:0485H         LINE#         354
  C:048AH         LINE#         355
  C:048DH         LINE#         358
  C:0490H         LINE#         359
  C:0495H         LINE#         360
  C:0498H         LINE#         361
  C:049BH         LINE#         362
  C:04A5H         LINE#         363
  C:04A8H         LINE#         364
  C:04ACH         LINE#         365
  C:04B1H         LINE#         366
  C:04B5H         LINE#         367
  C:04BAH         LINE#         368
  C:04BEH         LINE#         369
  C:04C3H         LINE#         370
  C:04C9H         LINE#         374
  -------         ENDPROC       KEYSCAN
  -------         PROC          KEYDOWN
  C:0622H         LINE#         377
  C:0622H         LINE#         378
  C:0622H         LINE#         379
  C:0625H         LINE#         380
  C:062BH         LINE#         381
  C:062BH         LINE#         382
  C:062EH         LINE#         383
  C:0633H         LINE#         384
  C:0633H         LINE#         385
BL51 BANKED LINKER/LOCATER V5.00                                                      05/05/2011  10:22:17  PAGE 9


  -------         ENDPROC       KEYDOWN
  -------         PROC          TIME0
  C:0352H         LINE#         390
  C:035AH         LINE#         392
  C:035CH         LINE#         393
  C:035EH         LINE#         394
  C:0361H         LINE#         395
  C:0364H         LINE#         396
  C:0366H         LINE#         398
  C:0385H         LINE#         399
  C:0399H         LINE#         400
  C:03B8H         LINE#         401
  C:03D1H         LINE#         403
  C:03D3H         LINE#         404
  -------         ENDPROC       TIME0
  -------         ENDMOD        FUNCTION2

*** WARNING L16: UNCALLED SEGMENT, IGNORED FOR OVERLAY PROCESS
    SEGMENT: ?PR?BUSYTEST?FUNCTION2

Program Size: data=35.1 xdata=0 code=1596
LINK/LOCATE RUN COMPLETE.  1 WARNING(S),  0 ERROR(S)
